:1000000011298030A100FE30AF200130AF207530C3
:10001000A7003030C628A101A117AF00AF08031D0B
:100020001328030114280130AF020310A20CA20C04
:10003000A20CC0302205403EAF07FE30AF202F0893
:10004000AF28A101A117AF00FE30AF202F08AF28C5
:10005000A401AA00AB01A01124080319A0150530C2
:10006000A3002730A900103041200330A900E83058
:100070004120A90164304120A9010A3041202A0809
:100080004828A8002B08A7002A08A600DA2026087E
:10009000A600A3030319A011240803195228230260
:1000A000031859282608031DA011A0195928303E0D
:1000B000AF280800A300240803190C292308AF2047
:1000C000A4035B28AD000611861183160611861164
:1000D0000F30860583122D08A0188C283E30A7000B
:1000E0008030C6203330AC00A0201330A700883009
:1000F000C620A0206430C520A0206430C520223056
:10010000AC00A02028308B200C308B2006308B20B8
:10011000A0142D088C282014AC00201C9A288611CD
:10012000033C031C9F289F200530A700DC30C6201D
:10013000031408002014FE3C0319AD288615201C6A
:10014000201006150F3086052C08F039860406119C
:10015000AC0E2018A0283230C5202D080C29A11B78
:10016000622883178001840AFF3E031DB2280C29F0
:10017000A901A800FF30A807031CA907031C0C292C
:100180000330A700DF30C620BA28A701E83EA6004A
:10019000A709FC30031CCF28A6070318CC28A60704
:1001A0000000A70FCC282618D528A61CD9280000A7
:1001B000D9280800AB01AA011030AC00270DAA0D08
:1001C000AB0D2808AA022908031C290FAB0203184B
:1001D000F0282808AA0729080318290FAB070310DD
:1001E000A60DA70DAC0BDE2826080C291030B00098
:1001F000A701A601AD0CAC0C031C04292808A60716
:1002000029080318290FA707A70CA60CAB0CAA0CEA
:10021000B00BFA282A080C29831383120313000059
:100220000800A00107309F00E03083168500FF30F2
:10023000860081138312850186012030840060309E
:10024000B220A03084005030B22020308400303002
:10025000B120C830B82001207730622062206220AF
:100260002E3062207030622069306220633062205C
:100270006230622061306220733062206930622017
:10028000633062202E3062206E3062206C3062203B
:100290000B30A900B830B92001204430622043302F
:1002A00062204630622031306220363062204E308B
:1002B00062204C3062204330622020306220622075
:1002C000563062202D306220323062200730A90083
:1002D000D030B92001204C306220443062205230AE
:1002E00062202030622061306220663062207230ED
:1002F00062206530622067306220653062206C3099
:100300006220653062206E30622086188D29851F3C
:100310008B2905148C290510852901205330622072
:1003200069306220673062206E3062206130622066
:1003300062206C306220203062207A3062206F3080
:100340006220653062206B306220653062206E3042
:10035000622036140512831605128312372AC30150
:100360003C03A500C90149082502031CC829EB214B
:10037000B61CC6294308A6004908A200A601A20A85
:100380000314A60DA20BC1292608C304C90FB32963
:10039000B2014308B100B20CB10CB20CB10CB20CFA
:1003A000B10CB20CB10C0F30B2053208AD003108FF
:1003B000AC00A9010A30A800F620B1002B08B20059
:1003C000B4014308B3000F30B3050030B405310861
:1003D0003307C3000800BA01B9010618002A01302A
:1003E000B820B90A0319BA0A0B303A02031CFF29D4
:1003F000031DFE29B9303902031CFF296C2DED299C
:100400009B30B8200618B614061CB610361C212ADC
:10041000440EB100B200F030B1050F30B205320821
:10042000A7003108A600A9013A30A800DA20BD00D3
:100430008030A1000230A2003D080D20FF30622074
:100440002A2A03013619013EB618013A031936115A
:10045000031D3615C40A85140130A900F430B920F3
:100460008510A901F030A8002808B9200800BB01B8
:10047000C4013612361ACF2ABA01B901061C512A14
:10048000B90A0319BA0A0130B820AF303A02031C86
:10049000502A031D4F2AC9303902031C502A6C2DE3
:1004A0003E2ABA01B9010618832AB90A0319BA0A01
:1004B0000A30B8203618772A39080B3A3A04031D57
:1004C000622A762A3908193A3A04031D692A8514E2
:1004D000762A39084B3A3A04031D702A8510762A89
:1004E0003908FA3A3A04031D762A6C2D822A113013
:1004F0003A02031C822A031D812A95303902031C0B
:10050000822A6C2D532A41303B02031C882A6C2D11
:10051000BB0A3A08031D902A65303902031C912A50
:100520003616361CCE2A3B0EB100B200F030B105B3
:100530000F30B2053208A7003108A600A9014130EA
:10054000A800DA20BD008030A10080302120533087
:10055000622069306220673062206E306220613034
:10056000622062206C30622020306220673062207E
:1005700065306220763062206F3062206E306220FB
:1005800064306220653062206E3062208030A100CD
:100590000230A2003D080D20FF3062203A2A361CAE
:1005A000F92A0120493062206E30622069306220D1
:1005B0007430622069306220613062206C306220C9
:1005C00069306220733062206530622072306220B0
:1005D000653062206E3062202E3062206220622000
:1005E0008030A100C03021201030A4005F305A209C
:1005F0005E2B0B30BD000130A2003D080B20A10195
:10060000B61D112B3B3041020318082BC10A102BD9
:10061000C1011730450203180F2BC50A102BC50165
:10062000152B4208C1004608C500051B252B4508AF
:10063000031D1D2B0C30C700242B0D304502031C5D
:10064000242B0C304502C700292B4508C700203059
:1006500062200A30470203182F2B2030622080309E
:10066000A100470828203A3062200230A400410847
:100670002920051B472B0C3045020318422B613003
:100680006220442B703062200E30BD00492B0F30A9
:10069000BD00410803190130031D0301B5001E30E0
:1006A000410203190130031D03013504B500013077
:1006B00086180301350403195E2B442D361E422D86
:1006C000EB210130C9000F30490203186A2BEB21DE
:1006D000C90F632B3611B611EB21EB21EB21B61CB0
:1006E000732B0514742B05101230C9001430490205
:1006F00003187D2BEB21C90F762BEB210730BC00B3
:10070000AF214308C200EB21361D872BB6150630FA
:10071000BC00AF214308C600EB21361D902BB61557
:100720000630BC00AF214308BE000330BC00AF213F
:100730004308C8000530BC00AF214308C0000830A2
:10074000BC00AF214308BF00EB21361DA82BB61516
:10075000361CAE2BB619AD2B36100120B619412D23
:100760008030A100803021200930A40020305A20A0
:100770008030A100C03021201030A40020305A2049
:1007800080302120A10101304802031DD52B4D30BE
:1007900062206130622062206E306220643062200C
:1007A00061306220673062204C2C02304802031D09
:1007B000E82B44306220693062206E306220733052
:1007C00062206430622061306220673062204C2CED
:1007D00003304802031DFD2B573062206F3062202A
:1007E000653062206E306220733062206430622097
:1007F00061306220673062204C2C04304802031DB7
:10080000142C443062206F3062206E3062206430DD
:100810006220653062207230622064306220613074
:100820006220673062204C2C05304802031D272CC3
:100830005630622072306220693062206A30622055
:100840006430622061306220673062204C2C0630B8
:100850004802031D3C2C5A30622061306220743003
:100860006220653062207230622064306220613024
:100870006220673062204C2C07304802031D4C2C4C
:100880005A3062206F3062206E3062206430622005
:1008900061306220673062208030A100C0302120AA
:1008A0003E0828202030622001304002031D672CC2
:1008B0006A306220613062206E30622075306220C2
:1008C000613062207230622069306220262D023051
:1008D0004002031D7C2C663062206530622062304D
:1008E0006220723062207530622061306220723086
:1008F000622069306220262D03304002031D8A2CBD
:100900006D3062206130622062207230622074306B
:100910006220262D04304002031D992C6130622094
:100920007030622072306220693062206C30622048
:10093000262D05304002031DA42C6D306220653049
:10094000622069306220262D06304002031DB12C42
:100950006A306220753062206E3062206930622019
:10096000262D07304002031DBE2C6A3062207530F0
:1009700062206C30622069306220262D08304002EF
:10098000031DD32C613062207530622067306220F5
:1009900075306220733062207430622075306220BE
:1009A00073306220262D09304002031DEA2C73307B
:1009B00062206530622070306220743062206530C1
:1009C00062206D30622062306220653062207230B9
:1009D0006220262D0A304002031DFD2C6F3062205C
:1009E0006B306220743062206F306220623062208F
:1009F0006530622072306220262D0B304002031DCC
:100A0000122D6E3062206F306220763062206530A9
:100A100062206D3062206230622065306220723068
:100A20006220262D0C304002031D262D64306220EA
:100A30006530622063306220653062206D30622054
:100A400062306220653062207230622009304002DC
:100A5000031D352D20306220273062208030A10018
:100A60000230A4003F082920412D2030622032307E
:100A70006220303062208030A1000230A4003F08A4
:100A80002920432D6C2D372A851F4B2D05128316E7
:100A9000051283124D2D8316051683129B30B82044
:100AA000410803190130031D0301B5000130861808
:100AB0000301350403195D2D0515851585140130D5
:100AC000A900F430B9200511851185100130A90065
:100AD0004A30B920C40A612B0120473062206530BA
:100AE000622062206E3062202030622073306220EB
:100AF00069306220673062206E306220613062208F
:100B000062206C306220203084006030B220A0303F
:100B100084005030B220203084003030B1200618DC
:100B2000B616061CB61203010618013EB61A013CA1
:100B3000031DA02DB70A0319B80A0130B820932D60
:100B40000301B61A0130013A0319B612031DB61695
:100B500003010618013EB61A013C031DB52DB70A64
:100B60000319B80A0130B820A82D03303802DE304E
:0C0B7000031937020318832D3614372AAE
:02400E00503F21
:00000001FF
